:103937000ECF0EBB0EA70E920E7C0E650E4D0E34EB
:103947000E190DFE0DE10DC40DA50D850D640D427B
:103957000D1E0CFA0CD40CAE0C860C5D0C330C0847
:103967000BDC0BB00B820B540B250AF50AC40A9328
:103977000A610A2F09FD09CA09960963092F08FC7C
:1039870008C808950861082E07FB07C8079607644B
:103997000733070206D206A206730645061705EA8D
:1039A70005BF059305690540051704F004C904A37D
:1039B700047E045A0437041503F403D303B40396AF
:1039C7000378035B033F0324030A02F002D702BF15
:1039D70002A80292027C02670253023F022C021ADB
:1039E700020801F701E601D601C701B801A9019C48
:1039F700018E018101740168015D01510146013C9D
:103A070001320128011F0115010D010400FC00F41A
:103A170000EC00E500DE00D700D000CA00C300BDFF
:103A270000B800B200AD00A700A2009E0099009464
:103A37000090008C008700840080007C007800756F
:103A47000072006E006B0068006500620060005D38
:103A5700005A0058005500530051004E004C004AD0
:103A670000480046004400430041003F003E003C40
:103A7700003A003900370036003500330032003194
:103A8700002F002E002D002C002B002A00290028D3
:103A9700002700260025002400230FA60FA00F995A
:103AA7000F920F8B0F840F7C0F740F6B0F620F58E1
:103AB7000F4E0F430F380F2C0F1F0F120F050EF766
:103AC7000EE80ED80EC80EB70EA50E930E800E6C1C
:103AD7000E580E420E2C0E150DFD0DE40DCB0DB13B
:103AE7000D950D790D5D0D3F0D200D010CE10CC0FD
:103AF7000C9E0C7C0C590C350C100BEA0BC40B9E5E
:103B07000B760B4F0B260AFD0AD40AAA0A800A5520
:103B17000A2A09FF09D409A8097C0950092508F9C7
:103B270008CD08A10875084A081E07F307C8079DAE
:103B370007730749072006F706CE06A6067E06572F
:103B47000630060A05E405BF059B057705540532CF
:103B5700051004EF04CE04AE048F0471045304353A
:103B6700041903FD03E203C703AD0394037B036357
:103B7700034B0334031E030802F302DE02CA02B634
:103B870002A30291027F026D025C024C023C022CEE
:103B9700021D020E020001F201E401D701CA01BEB3
:103BA70001B101A6019A018F0185017A01700166B1
:103BB700015D0153014A0141013901310129012107
:103BC70001190112010B010400FD00F700F000EAE2
:103BD70000E400DE00D900D300CE00C900C400BF56
:103BE70000BA00B500B100AD00A800A400A0009C79
:103BF700009900950091008E008A0087008400815B
:103C0700007E007B00010C01010502011E030A96DC
:103C170004013205050506006407010108000009D3
:103C2700015A0A01040B00030E01010F00011200E3
:103C37006413010114013C1501FA1664FA17FFFF1A
:103C47001D00072000072400022632962701012CB9
:103C5700000130030332010333000235FFFF36034F
:103C6700073CFFFF3DFFFF180002191E461A00021E
:0F3C77001B00022D32C82E00012F013CFAFAFA71
:10004800E50C901FEDF8282873803475E700A2109E
:10005800B34008E5B54408F5B58006E5B554F7F5AD
:10006800B575E710801975E700A210B34008E5B52B
:0F0078004402F5B58006E5B554FDF5B575E71002
:091FED0002005102005302006ED3
:100087002290083CE0900042F090083DE090004943
:10009700F090083EE090004AF090083FE090004D55
:1000A700F0900840E090004EF0900841E090005139
:1000B700F0900842E0900052F0900843E090005D15
:1000C700F0900844E090005FF0900845E0900063EE
:1000D700F0900846E0900065F0900847E0900066D1
:1000E700F0900848E0900067F0900849E0900068B9
:1000F700F090084AE090006BF090084BE090006C9D
:10010700F090084CE090006EF090084DE090006F82
:10011700F090084EE090007BF090084FE090007C54
:10012700F0900850E090007DF0900851E090007E3C
:10013700F0900852E090007FF0900853E090008024
:10014700F0900854E0900081F0900855E09000820C
:10015700F0900856E0900084F0900857E0900085F2
:10016700F0900858E0900086F0900859E0900087DA
:10017700F090007BE090002BF090007CE090002C4A
:10018700F090007DE090002DF090007EE090002E32
:10019700F090007FE090002FF0900080E09000301A
:1001A700F0900081E0900031F0900082E090003202
:1001B700F0900084E0900027F0900085E090002800
:1001C700F0900086E0900029F0900087E090002AE8
:1001D700F07441900110F07469900111F0747390FC
:1001E7000112F07469900113F0746E900114F074A9
:1001F70020900115F07441900116F07437900117A3
:10020700F07435900118F07430900119F07445902E
:10021700011AF0742090011BF0743590011CF074E2
:100227005390011DF0747090011EF09003FFE09051
:10023700043FF022900839E0FEA3E0FF7463BE009C
:1002470010D39F400C903C0B12001EE493F599804D
:1002570012900839E0FEA3E0FF903C0B12001EE469
:1002670093F59990083912000E900839E0FEA3E043
:10027700FF747B6F4E700375670022A206B34016AA
:10028700900125E0700C900126E07006900127E0B0
:1002970060028002C206900125E0B4300F9001266B
:1002A700E0B44708900127E0643B60028004D2076E
:1002B7008002C207E549B40102800302038D900062
:1002C7007BE090002BF090007CE090002CF09000F9
:1002D7007DE090002DF090007EE090002EF09000E1
:1002E7007FE090002FF0900080E0900030F09000C9
:1002F70081E0900031F0900082E0900032F09000B1
:1003070084E0900027F0900085E0900028F09000AE
:1003170086E0900029F0900087E090002AF0900096
:1003270064E0B40117900000740FF0A374FFF0901D
:100337000002E4F0A3F07402900064F0900064E01F
:10034700B40341900002E0FEA3E0FF900000E0FC50
:10035700A3E0FD1200037410123E567408123E48C3
:10036700EF900063F0EF700674FF900063F0740085
:10037700900064F0900001E0900049F0900000E0E8
:1003870090004AF0800990006CE070037549017E87
:10039700897FE7900042E08E048F05FF123E388C7C
:1003A700338D3490004EE075F0FAA4FFAEF0900064
:1003B7004DE08E048F05FF123E388C378D38900044
:1003C7003AE0F54F900037E0FE900054E0B506188C
:1003D700900036E0FE900053E0B5060C900035E043
:1003E700FE900044E06E606F900054E0700690004D
:1003F70053E060067400900044F0900054E0B402AB
:10040700089000337401F08005900033E4F0900009
:1004170053E0B402089000347401F0800590003472
:10042700E4F0900053E06006900034E0600280053D
:10043700754F048003754F05E54AB54902D20A9006
:100447000053E0900036F0900054E0900037F090B1
:100457000044E0900035F07401900089F07400903A
:10046700008AF0740090008BF0740090008CF07498
:100477000190008DF0740090008EF0740090008F52
:10048700F07401900090F07400900091F074009067
:100497000092F07400900093F07401900094F0744F
:1004A70000900095F07400900096F074019000970A
:1004B700F07400900098F07400900099F074009028
:1004C700009AF0740190009BF0740090009CF07407
:1004D7000090009DF0740190034DF0740090034E5E
:1004E700F0740090034FF07400900350F074019083
:1004F7000351F07400900352F07400900353F074AA
:100507000190038DF0740190038EF0740090038FB7
:10051700F07400900390F07401900391F0740090D0
:100527000392F07400900393F074009003CDF0747D
:10053700019003CEF074009003CFF074009003D0C5
:10054700F074019003D1F074009003D2F07400901E
:1005570003D3F0740090040DF0740090040EF0744F
:100567000090040FF07400900410F07401900411CF
:10057700F07400900412F07400900413F07400906B
:10058700044DF0740090044EF0740190044FF07421
:1005970001900450F07400900451F07400900452DC
:1005A700F07400900453F012201722C293C294C231
:1005B70091C292C287755200755300C203E5B554C4
:1005C700FBF5B5754405E54404F54590003AE0F5BB
:1005D7004F900026E4F0C205900038E4F0E5B554EA
:1005E700FEF5B5900026E4F0755100C28E758D00BA
:1005F700758B00754100752600752500D28EC29651
:10060700C295C2A0E5B554EFF5B5E5B554DFF5B52C
:10061700E5B554F7F5B5E5B554FDF5B522755900BF
:10062700755800AE58AF597462BE00039F5003025D
:1006370006E1903C0B12001EE493900039123E6EC7
:100647000FBF00010EE0FC903C0B12001EECFEE415
:1006570093FFEEC39F5026AE58AF590FBF00010E50
:10066700903C0B12001EAE58AF59E493FC903C0B24
:1006770012001EE493900039123E6EECF0AE58AFB4
:1006870059903C0B12001EE493900039123E6EE025
:10069700FC903C0D12001EECFCE493FDECD39D4056
:1006A70019903C0D12001EE493FC903C0B12001EA7
:1006B700E493900039123E6EECF0AE58AF597402D5
:1006C7002FFF50010E8E588F597859740126F65016
:1006D7000418E436F6400302062A227559007558B5
:1006E70000AE58AF597417BE00039F50030207AFFF
:1006F700903C6E12001EE493900039123E6E0FBFBD
:1007070000010EE0FC903C6E12001EECFEE493FF2D
:10071700EEC39F5026AE58AF590FBF00010E903C55
:100727006E12001EAE58AF59E493FC903C6E120057
:100737001EE493900039123E6EECF0AE58AF59901C
:100747003C6E12001EE493900039123E6EE0FC905E
:100757003C7012001EECFCE493FDECD39D40199015
:100767003C7012001EE493FC903C6E12001EE49352
:10077700900039123E6EECF0AE58AF5974126F4EBE
:100787007006755918755800AE58AF5974022FFF87
:1007970050010E8E588F597859740126F650041857
:1007A700E436F640030206E8221206241206E22285
:1007B7000542220541220543C2CF2290F800E49367
:1007C7006406600280FE75840175A70075FF80903E
:1007D700083BE4F075C91075A70F75A1C775A70089
:1007E70075D90075CEFF75A70F75F1FE75F2FF7508
:1007F700F33775F47875A4BA75A5FF75A60775AEB6
:100807000075AFFF75D48175D5FF75D6FF75D7FF16
:10081700C296C295C2A0E5B554EFF5B5E5B554DF6C
:10082700F5B5E5B554F7F5B5E5B554FDF5B575A7D7
:100837000075A20175A14775F80975BC0175BE045D
:1008470075BD6C75BE0775BDA075BE0875BD017514
:10085700BC0075BB1875BC2075BA0875E88075D1E2
:100867001375A70F75E10575E20075C74075970009
:10087700759780740A123E287597C0E597542070C3
:100887000280F8758F0275A700D2AF75980075A919
:100897000C75A70F75AB4375ADFB75AC1E75A7003F
:1008A700758911758E00758C00758A00D2A9D28C56
:1008B700758D00758B00D2ABD28E75CD0075CC00CF
:1008C70075CA0075CB00D2ADC2CFD2CA7591047577
:1008D70092007593CD75EF0675D94075CF019008D5
:1008E70039E4F0A3F0756700756800C299D206C2B3
:1008F7000B1205B274C8F50975080012214D75A7CA
:100907000FE5FC900015F0E5FB900016F0E5FA9076
:100917000017F0E5F9900018F075A70090F800E4CB
:1009270093F55712226C1227A690F807E4939000CC
:1009370022F0900022E04408900022F0900022E08C
:1009470054FE900022F0120088900859E09001258B
:10095700F090085AE0900126F090085BE09001279C
:10096700F0900125E0700C900126E07006900127B9
:10097700E060028004C2068002D206754901754A0A
:10098700017403900036F01207B07400900064F011
:10099700740090006DF01202827406900008F074E3
:1009A70000900009F0740290000AF090F802E493B6
:1009B70090000BF090F803E49390000CF090F8048B
:1009C700E49390000DF0740590000EF0740590000C
:1009D7000FF07403900010F07406900011F0740289
:1009E700900012F090F805E493900013F090F80649
:1009F700E493900014F0740090001CF074009000D1
:100A07001DF0740090001EF0740090001FF0740039
:100A1700900020F07400900021F074FF900023F004
:100A2700A2B6B39200A2B3B39201756D00743A9067
:100A37000739F074FD90073AF0C20A900024E4F0F9
:100A4700754B00752400752300753E00752A0075E7
:100A57002900753F007546007547007545017555B6
:100A6700007554007556CD754800753B00753C0000
:100A7700753D00753A00753900754E009000047495
:100A8700FDF0A374E8F0900024E4F074649000256E
:100A9700F0754200E5B554BFF5B5E5B5547FF5B53A
:100AA700C2A1C2A2C297122120C203D2B0D2B7D22A
:100AB700A7D2A6D2B1D2A37E017F0090004AE0124E
:100AC7003E56900049E02FFF50010E900000EEF0D7
:100AD700A3EFF0EFD394FFEE940F4007900000E4EC
:100AE700F0A3F0900063E0700674FF900063F0D20B
:100AF7009CD2EC75CF01A298B34005C298122B5235
:100B0700E5676006A299B3B340028005C299122F28
:100B170068E56864016005E568B4040280D5E542CC
:100B2700D39405400CE54BC394C85002054B75425E
:100B370000E556C394F0501A785412003FAE54AFF4
:100B470055EFD394E8EE94034008055675550075A4
:100B57005400C28E7E047F00E541123E56E58D7536
:100B6700F004A4FDACF0EF2DFDEE3CFCE58B75F039
:100B77004084FF7E00ED2FFFEC3EFE8E258F26D2B0
:100B87008EA2B6300001B35003020CDDA2B63000CE
:100B970001B35003020CDDA2B640730546A20B4019
:100BA7000575FFA0D20BE5B54401F5B5900025E426
:100BB700F0900042E0C395465052E5264525600F68
:100BC7007C897DE7AE25AF26123C868E238F24AE27
:100BD70023AF24E53E2FFF50010E7401123E488ECD
:100BE700238F2485243E754601C28E758D00758B33
:100BF70000754100D28E7403BE00039F500690001B
:100C0700267401F0E56DB40D03756D00D200A2B630
:100C1700B35003020CDD900025E4F0C200900056AB
:100C2700E060067508011230A9900059E06006756A
:100C370008021230A9A203B34008E5B54440F5B550
:100C47008006E5B554BFF5B5900044E06008E5B50A
:100C57004480F5B58006E5B5547FF5B5900034E0DE
:100C6700B40104D2A18002C2A1900033E0B4010410
:100C7700D2A28002C2A2A205B34004D2978002C2C8
:100C87009790000EE0FE90000BE0C39E4009900095
:100C97000BE0D39408400974FB900024F01205B2CE
:100CA70090000CE0601590000CE0FE90000AE06EEA
:100CB700600974FC900024F01205B290000DE0600A
:100CC7001590000DE0FE90000FE06E600974FE9035
:100CD7000024F01205B2C2CA7E017F00E543123E2E
:100CE70056E5CD2FFF50010E8E278F28D2CA9000D0
:100CF70067E0B40148900004E0FCA3E0FDEFC39D6A
:100D0700EE9C4039B204E52A45296013A204B3409A
:100D170008E5B54404F5B58006E5B554FBF5B5908F
:100D27000004E0FEA3E0FF900006E0FCA3E0FDEF77
:100D37002DFDEE3CFC900004ECF0A3EDF0A2B330E7
:100D47000101B35003020E7DA2B3300101B350037A
:100D5700020E7DA2B35003020E760547A20B400593
:100D670075FFA0D20BE5B54401F5B5900025E4F079
:100D770090004DE0C395474003020E74E5284527D0
:100D8700600F7CEA7D60AE27AF28123C868E298FE4
:100D97002AAE29AF2A90004EE0123E5674FF8E0409
:100DA7008F05FF123E388C298D2AE53F2DFD500116
:100DB7000C74018C068D07123E488E298F2A852ACE
:100DC7003FA205B340157464123E56900052E08E60
:100DD700048F05FF123E388C298D2A754701900034
:100DE70004E0FEA3E0FFAC27AD2812000390000447
:100DF700EEF0A3EFF07AFF7BFF900066E08A048BAA
:100E070005FF123E38AE27AF28EDD39FEC9E402357
:100E1700900066E0123E5674828E048F05FF123EE4
:100E270038900068E0FF123E38900006ECF0A3ED22
:100E3700F0802DAE27AF2874828E048F05FF123EF7
:100E470038900066E08C068D07123E56900068E0E9
:100E57008E048F05FF123E38900006ECF0A3EDF0EC
:100E6700C2CA75CD0075CC00754300D2CAD201A2A3
:100E7700B3B34002C201900026E0B40107E548C3BE
:100E87009406400302149DE551901FF6F828287335
:100E9700900044E0C394024003020FEBE544D3946F
:100EA700015003020FEBE54475F040A4FFAEF0904C
:100EB70002FD12001EE0C3953C5018E54475F04052
:100EC700A4FFAEF09002FC12001EE0F52E752D0077
:100ED700020FEBE54475F040A4FFAEF09002FB1261
:100EE700001EE0C3953C4003020F87E54475F040C0
:100EF700A4FFAEF09002FC12001EE54475F040A47A
:100F0700FFAEF0E0FC9002FA12001EECFEE0FFEEEE
:100F1700C39FFEE5448E0475F040A4FFAEF0900237
:100F2700FB12001EE0F404253C8C0088F0A4FFAE01
:100F3700F0E5448F048E0575F040A4FFAEF09002F3
:100F4700FD12001EE54475F040A4FFAEF0E0FA90F4
:100F570002FB12001EEAFEE0FFEEC39FFECDCCCDE2
:100F67008E07123E38E54475F040A4FFAEF09002BC
:100F7700FA12001EE02DFD50010C8C2D8D2E806481
:100F8700E54475F040A4FFAEF09002FA12001EE5AA
:100F97004475F040A4FFAEF0E0FC9002F912001E89
:100FA700ECFEE0FFEEC39F853CF0A4FFAEF0E54406
:100FB7008F048E0575F040A4FFAEF09002FB12007F
:100FC7001EE0FECDCCCD8E07123E38E54475F040CD
:100FD700A4FFAEF09002F912001EE02DFD50010CA7
:100FE7008C2D8D2E75510102149D900044E0C39401
:100FF70002400302119F90003AE0D3954450030248
:101007001147E54475F040A4FFAEF09003031200CA
:101017001EE0C3953C5018E54475F040A4FFAEF0C0
:1010270090030212001EE0F52C752B00021147E514
:101037004475F040A4FFAEF090030112001EE0C318
:10104700953C40030210E3E54475F040A4FFAEF081
:1010570090030212001EE54475F040A4FFAEF0E0D5
:10106700FC90030012001EECFEE0FFEEC39FFEE5BE
:10107700448E0475F040A4FFAEF090030112001EE9
:10108700E0F404253C8C0088F0A4FFAEF0E5448F23
:10109700048E0575F040A4FFAEF090030312001E06
:1010A700E54475F040A4FFAEF0E0FA9003011200AA
:1010B7001EEAFEE0FFEEC39FFECDCCCD8E07123EAB
:1010C70038E54475F040A4FFAEF090030012001E0F
:1010D700E02DFD50010C8C2B8D2C8064E54475F0C0
:1010E70040A4FFAEF090030012001EE54475F040E7
:1010F700A4FFAEF0E0FC9002FF12001EECFEE0FF42
:10110700EEC39F853CF0A4FFAEF0E5448F048E0547
:1011170075F040A4FFAEF090030112001EE0FECD73
:10112700CCCD8E07123E38E54475F040A4FFAEF0F3
:101137009002FF12001EE02DFD50010C8C2B8D2C10
:10114700E544B40123E54FD39401401CE54804D39B
:1011570095444014E53CC39405500D90034AE0A81C
:1011670029B80006952A40028003754402E544B574
:101177004F2290003AE0D395444019E54475F0407A
:10118700A4FFAEF090030212001EE0A823B80006E9
:10119700952440028002054F75510202149D90006C
:1011A70044E0B4022AE54475F040A4FFAEF0900392
:1011B7000212001EE0F52C752B00E54475F040A4E3
:1011C700FFAEF09002F912001EE0F52E752D00908B
:1011D7000044E0B4030F90003CE0F52C752B00753C
:1011E7002E00752D0075510302149DE54475F040DE
:1011F700A4FFAEF090030B12001EE0C3954B400313
:101207000212C7900033E07036E544D394014029B9
:10121700AE23AF24AC2DAD2EEDD39FEC9E401AE547
:101227004475F040A4FFAEF090030912001EE0A839
:1012370029B80005D3952A5002800215448034E569
:1012470044D394024029AE23AF24AC2DAD2EEDD369
:101257009FEC9E401AE54475F040A4FFAEF0900362
:101267000912001EE0A829B80005D3952A5002806C
:10127700021544E544B54537E544C3954F5030E57D
:101287004804D395444028AE23AF24AC2BAD2CEFB4
:10129700D39DEE9C4019E54475F040A4FFAEF09055
:1012A700030A12001EE0A829B80006952A4002800A
:1012B700020544C287E54465456005C203754B00D6
:1012C70075510402149DE54475F040A4FFAEF090FB
:1012D700030512001EE0B40117E54475F040A4FFB2
:1012E700AEF090030B12001EE0240AC3954B400397
:1012F70002139D753064752F00A203B3500B900045
:101307004BE02405C3953C400302139DE54475F06B
:1013170040A4FFAEF090030812001EE0C3953C40C6
:1013270064E54475F040A4FFAEF090030712001E79
:10133700E54475F040A4FFAEF0E0FC900306120010
:101347001EECFEE0FFEEC39F853CF0A4FFAEF0E588
:10135700448F048E0575F040A4FFAEF09003081289
:10136700001EE0FECDCCCD8E07123E38E54475F069
:1013770040A4FFAEF090030612001EE02DFD5001C1
:101387000C8C2F8D30AE23AF24AC2FAD30EFD39D17
:10139700EE9C4002D20375510502149DE544B40149
:1013A70009900044E0C39402400302147190034380
:1013B700E0D3953C5003021471900341E0C3953C80
:1013C7005040900342E0FE900340E0F4042EFE906C
:1013D7000341E0F404253C8E0088F0A4FFAEF090B2
:1013E7000343E0FC900341E0F4042C8E048F05FFD7
:1013F700123E38900340E02DFD50010C8C2B8D2CB4
:10140700802C900340E0FE90033FE0F4042E853CDF
:10141700F0A4FFAEF0900341E08E048F05FF123E6B
:101427003890033FE02DFD50010C8C2B8D2CE544AB
:10143700C3954F5030E54804D395444028AE23AFB9
:1014470024AC2BAD2CEFD39DEE9C4019E54475F0F1
:1014570040A4FFAEF090030A12001EE0A829B800CE
:1014670006952A40028003754402900033E0B401D8
:1014770006E544640160028003754402E54465455E
:101487006005C203754B00E54BD3940A40059000F5
:0614970038E4F07551007D
:101FF600020E97020FF10211A50211F20212CD0292
:0220060013A322
:10149D0090003BE02402A823B80007D39524400216
:1014AD00C203900026E0B40109900044E0C3940308
:1014BD004003021631900033E0600302157AE544D3
:1014CD00D39401403A900038E07034E54475F04013
:1014DD00A4FFAEF09002FF12001EE0A823B8001F7B
:1014ED00D39524401AE54475F040A4FFAEF0900367
:1014FD000A12001EE0A829B80005D3952A500280D3
:10150D00021544E544D39401402FE54475F040A401
:10151D00FFAEF09002FD12001EE0C3953C501AE59F
:10152D004475F040A4FFAEF090030912001EE0A830
:10153D0029B80005D3952A500280021544E544D3FD
:10154D0094014022E54804C39544501AE54475F0D2
:10155D0040A4FFAEF090030912001EE0A829B800C8
:10156D0005D3952A500280021544021626E544D370
:10157D009402403A900038E07034E54475F040A490
:10158D00FFAEF09002FF12001EE0A823B8001FD39B
:10159D009524401AE54475F040A4FFAEF090030A7F
:1015AD0012001EE0A829B80005D3952A500280022A
:1015BD001544E544D39402402FE54475F040A4FF53
:1015CD00AEF09002FD12001EE0C3953C501AE544AA
:1015DD0075F040A4FFAEF090030912001EE0A8299B
:1015ED00B80005D3952A500280021544E544D394E2
:1015FD00024022E54804C39544501AE54475F04075
:10160D00A4FFAEF090030912001EE0A829B8000552
:10161D00D3952A500280021544E54465456005C204
:10162D0003754B0090004BE0D3953C500990003F63
:10163D00E0C3953C5002C203900044E070030218D1
:10164D00AEA2A5B34008A2A4B34003021897AE31D1
:10165D00AF327441D39F749C9E4005783112003F88
:10166D00AE31AF32EFB48806EEB413028003021828
:10167D0072A2A55003021728900044E0B401109007
:10168D00003AE0D3954F4002054FE54404F54590EF
:10169D000044E0B40256E54475F040A4FFAEF0906E
:1016AD00030B12001EE0C3954B504190003AE0D35E
:1016BD0095444021E54804D395444019E54475F01F
:1016CD0040A4FFAEF09002FF12001EE0A823B80068
:1016DD0006952440028002054485444FE544654546
:1016ED006005C203754B00E54404F545900044E0E8
:1016FD00B4032890003AE0D395444008E54804D35C
:10170D00954450028002054485444FE5446545608B
:10171D0005C203754B00E54404F545A2A450030230
:10172D001872900044E0B40173900033E0703AE514
:10173D0044D394014029E54475F040A4FFAEF090E8
:10174D00030912001EE0A829B8000FD3952A400AFC
:10175D001544754B0085444F800385444F800375B8
:10176D004F01E54404F5458033E544D39402402907
:10177D00E54475F040A4FFAEF090030912001EE0A1
:10178D00A829B8000FD3952A400A1544754B00853A
:10179D00444F800385444F8003754F02900044E011
:1017AD00D394015003021866E54475F040A4FFAED2
:1017BD00F090030B12001EE0C3954B400302186618
:1017CD00900033E07041E544D394014034E5447515
:1017DD00F040A4FFAEF09002FC12001EE0A823B86A
:1017ED00001FD39524401AE54475F040A4FFAEF0D8
:1017FD0090030912001EE0A829B80005D3952A50C0
:10180D000280021544803FE544D394024034E54400
:10181D0075F040A4FFAEF09002FC12001EE0A8236C
:10182D00B8001FD39524401AE54475F040A4FFAECF
:10183D00F090030912001EE0A829B80005D3952ADF
:10184D0050028002154485444FE54465456005C24C
:10185D0003754B00E54404F545E548B40704054E12
:10186D008003754E0090006CE0B4010EAE31AF32C6
:10187D00EF64407005EE649C6002800EA2A54003EB
:10188D00754901A2A44003754902A2A5B3B3500640
:10189D00A2A4B3B34002800675320075310002195F
:1018AD009CA2A5B34008A2A4B34003021988AE318F
:1018BD00AF327441D39F749C9E4005783112003F26
:1018CD00AE31AF32EFB48806EEB4130280030219C5
:1018DD0088A2A5406F900053E0605A900034E0B4A8
:1018ED000107900034E4F080069000347401F0900C
:1018FD000034E07005754F048003754F059000347A
:10190D00E0B40104D2A18002C2A1E544B4051AE5F8
:10191D004475F040A4FFAEF090030912001EE0A83C
:10192D0029B80005D3952A50028008754404C203D6
:10193D00754B008003754F05E548B40704054E80CF
:10194D0003754E00A2A44033900054E06021900036
:10195D0033E0B40107900033E4F080069000337457
:10196D0001F0900033E0B40104D2A28002C2A2E5DE
:10197D0048B40704054E8003754E00A2A5B3B350BD
:10198D0006A2A4B3B340028006753200753100E59E
:10199D0049654A600690006DE06002802CE5499033
:1019AD002008F828287380121227A6800D1228917E
:0A19BD00800812297C8003122A67BB
:0F2008000219B30219B50219BA0219BF0219C49D
:1019C70012008812028285494A741B900024F0E5B0
:1019D70048C394065005E544B54503021AB2C2034D
:1019E700E54475F040A4FFAEF090030D12001EE031
:1019F70030E003D38001C39296E54475F040A4FF1D
:101A0700AEF090030E12001EE030E003D38001C356
:101A17009295E54475F040A4FFAEF090030F1200D5
:101A27001EE030E003D38001C392A0E54475F04087
:101A3700A4FFAEF090031012001EE030E003D38045
:101A470001C39208E54475F040A4FFAEF09003117E
:101A570012001EE030E003D38001C39209E548B4C9
:101A67000206E544640360028002C209E548B40146
:101A770006E544640260028004D2A0C209E548B4C6
:101A8700010BE544B40106E54F640160028002C220
:101A970009854445AE29AF2A7405BE00039F500748
:101AA700E53CD3940550028002D287E548D39405DC
:101AB7005003021C42C203E544D394015003021BA6
:101AC70070E54475F040A4FFAEF090030912001EC4
:101AD700E0A829B80007D3952A40021544E54465D4
:101AE700457003021B6DE54475F040A4FFAEF0900E
:101AF700030D12001EE030E003D38001C39296E588
:101B07004475F040A4FFAEF090030E12001EE030C3
:101B1700E003D38001C39295E54475F040A4FFAE7E
:101B2700F090030F12001EE030E003D38001C39250
:101B3700A0E54475F040A4FFAEF090031012001E1C
:101B4700E030E003D38001C39208E54475F040A478
:101B5700FFAEF090031112001EE030E003D38001C6
:101B6700C39209854445021C42E548B406419000EA
:101B770097E030E003D38001C39296900098E0305D
:101B8700E003D38001C39295900099E030E003D33E
:101B97008001C392A090009AE030E003D38001C394
:101BA700920890009BE030E003D38001C39209E5DF
:101BB70048B40741900090E030E003D38001C3921E
:101BC70096900091E030E003D38001C39295900096
:101BD70092E030E003D38001C392A0900093E030FD
:101BE700E003D38001C39208900094E030E003D370
:101BF7008001C39209E548B40841900089E030E0CC
:101C070003D38001C3929690008AE030E003D3802B
:101C170001C3929590008BE030E003D38001C3921B
:101C2700A090008CE030E003D38001C392089000BD
:101C37008DE030E003D38001C3920990005DE0603E
:101C470058E53C75F00284FF7E0090013912001EB2
:101C5700E0F54CE53D75F00A84FF7E0090023912ED
:101C6700001EE0F54DE54C254DD39464400BE54C43
:101C7700254DC39464F54C8003754C00E54C75F015
:101C87000284FF7E008F4CEFC394335007EF24CDBF
:101C9700F54C8003754CFF801CE53C75F00284FF12
:101CA7007E0090013912001EE075F00284FF7E006D
:101CB700EF24CDF54CE595C3954C4004C2938002C3
:101CC700D293A203B34005E548B407037556CDE5A3
:101CD70095C395564004C2948002D294E53C75F0B2
:101CE7000284FF7E0090016B12001EE075F00284F3
:101CF700FF7E00EF24CDF552E595C395525006A21D
:101D070008B3B340028004D2918002C291E56DC34B
:101D1700940D501DE56D75F00284AFF07E00EF4E17
:101D270070051232EF800AA2EDB34005C2ED123200
:101D3700EFE54ED394045003021ED275CF01C29330
:101D4700AE31AF327488D39F74139E4005A2A5B3FA
:101D57004014AE31AF327488D39F74139E4005A2EE
:101D6700A4B340028048783112003FAE31AF32EF62
:101D7700B4883BEEB41337A2A5B3500990003AE0FC
:101D8700D395445002800405448011A2A5B350089E
:101D970090003AE0654460028002D203A2A4B350E7
:101DA70007E544D39401500280041544C203A2A559
:101DB700B3B35006A2A4B3B34002800675320075D0
:101DC7003100E54465457003021E54E54475F04053
:101DD700A4FFAEF090030D12001EE030E003D380A5
:101DE70001C39296E54475F040A4FFAEF090030E50
:101DF70012001EE030E003D38001C39295E54475DD
:101E0700F040A4FFAEF090030F12001EE030E00395
:101E1700D38001C392A0E54475F040A4FFAEF090D3
:101E2700031012001EE030E003D38001C39208E5DF
:101E37004475F040A4FFAEF090031112001EE0308D
:101E4700E003D38001C39209C294854445A20340AD
:101E5700057556CD80037556FFE595C39556400425
:101E6700C2948002D294E53C75F00284FF7E009014
:101E7700016B12001EE075F00284FF7E00EF24CD97
:101E8700F552E595C395525006A208B3B3400280B8
:101E970004D2918002C291E53C75F00284FF7E0076
:101EA70090019D12001EE075F00284FF7E00EF2472
:101EB700CDF553E595C395535006A209B3B3400238
:101EC7008004D2928002C292021D42A20BB3500D2F
:101ED700AE25AF2674E8C39F74039E400280057544
:101EE700FFA0D20BAE25AF26EFD39420EE944E5031
:101EF70003021FC11205B2C28E758D00758B007566
:101F07004100D28EC2037555007554007556CD75C4
:101F17004405752400752300754600754B00E5B52B
:101F270054BFF5B5900044E06008E5B54480F5B5C9
:101F37008006E5B5547FF5B5900034E0B40104D2CE
:101F4700A18002C2A1900033E0B40104D2A28002B2
:101F5700C2A2A205B34004D2978002C2979000564E
:101F6700E060067508011230A9900059E060067517
:101F770008021230A990000474FDF0A374E8F0E59C
:101F87006DB40D03756D00752600752500758D0000
:101F9700758B00754100900025E0C39403500890AD
:101FA7000025E004F080067403900025F0900025DA
:101FB700E0B40306E5B554FEF5B5AE27AF28EFD379
:101FC7009410EE9427401CC2CA75CD0075CC0075DD
:101FD7002800752700D2CA754300752A00752900A5
:061FE700754700020AFA32
:103D6700000001000132016401960196020002126F
:103D770002240200020003000340038003C0040082
:103D87000440048004C00500060006000600060083
:103D9700060006000600060000FF013101630195D9
:103DA70001FF01FF0211022302FF02FF02FF033F8F
:103DB700037F03BF03FF043F047F04BF04FF05FF26
:103DC70006FF06FF06FF06FF06FF06FF06FF06FFC4
:10201700900042E090083CF0900049E090083DF0C5
:1020270090004AE090083EF090004DE090083FF0A5
:1020370090004EE0900840F0900051E0900841F089
:10204700900052E0900842F090005DE0900843F065
:1020570090005FE0900844F0900063E0900845F03E
:10206700900065E0900846F0900066E0900847F021
:10207700900067E0900848F0900068E0900849F009
:1020870090006BE090084AF090006CE090084BF0ED
:1020970090006EE090084CF090006FE090084DF0D3
:1020A70090007BE090084EF090007CE090084FF0A5
:1020B70090007DE0900850F090007EE0900851F08D
:1020C70090007FE0900852F0900080E0900853F075
:1020D700900081E0900854F0900082E0900855F05D
:1020E700900084E0900856F0900085E0900857F043
:1020F700900086E0900858F0900087E0900859F02B
:10210700900125E090085AF0900126E090085BF0D6
:10211700900127E090085CF022900839E4F0A3F0E2
:10212700755D00755C00756700756800C20DD20E9D
:1021370075610075600075633C756200756E0075AA
:102147006F00756C0022750B00750A00AE0AAF0BA5
:10215700AC08AD09EDC39FEC9E401674FF123E28F4
:1021670075CF01780B740126F6500418E436F65043
:10217700DB22C2AF75D900758F0375B7A575B7F1A7
:1021870090F800E4F0758F0175B7A575B7F1E557BD
:1021970090F800F075B7A575B7F190F801E4F07500
:1021A700B7A575B7F1900878E090F802F075B7A574
:1021B70075B7F190087CE090F803F075B7A575B78F
:1021C700F1900879E090F804F075B7A575B7F1902C
:1021D700087AE090F805F075B7A575B7F190087B18
:1021E700E090F806F075B7A575B7F190087DE09017
:1021F700F807F0758F0075D940D2AF2290083BE001
:10220700B4AB61C2AF75D90075B62275F522758F6B
:102217000375B7A575B7F1740090F600F0758F01D7
:10222700755900755800AE58AF59743BBE00279FCB
:10223700402475B7A575B7F190083C12001EE0FC65
:1022470090F60012001EECF07859740126F650043F
:1022570018E436F650D0758F0075F51175B62075F0
:10226700D940D2AF22C2AF75D90075F52275590092
:10227700755800AE58AF59743BBE00229F401F905F
:10228700F60012001EE493FC90083C12001EECF0CE
:102297007859740126F6500418E436F650D575F5CA
:1022A7001175D940D2AF2290083BE0B4AA0280034F
:1022B7000223EBC2AF75D90075B62275F522758F6B
:1022C7000375B7A575B7F1740090EE00F075B7A563
:1022D70075B7F1740090F000F075B7A575B7F17494
:1022E7000090F200F075B7A575B7F1740090F4008F
:1022F700F0758F01755900755800AE58AF5974FFC6
:10230700C39F74019E402475B7A575B7F190003936
:1023170012001EE0FC90EE0012001EECF0785974DB
:102327000126F6500418E436F650CF755900755853
:1023370000AE58AF5974FFC39F74019E402475B710
:10234700A575B7F190023912001EE0FC90F000125B
:10235700001EECF07859740126F6500418E436F69E
:1023670050CF755900755800AE58AF5974FFC39FC9
:1023770074019E402475B7A575B7F1900439120012
:102387001EE0FC90F20012001EECF0785974012652
:10239700F6500418E436F650CF755900755800AE5C
:1023A70058AF5974FFC39F74019E402475B7A57534
:1023B700B7F190063912001EE0FC90F40012001EDF
:1023C700ECF07859740126F6500418E436F650CF2D
:1023D700758F0075F51175B62075D940D2AF743A6F
:1023E700900739F02290083BE0B4AA028003022547
:1023F70029C2AF75D90075B62275F522758F037599
:10240700B7A575B7F1740090E600F075B7A575B775
:10241700F1740090E800F075B7A575B7F1740090F6
:10242700EA00F075B7A575B7F1740090EC00F07588
:102437008F01755900755800AE58AF5974FFC39F87
:1024470074019E402475B7A575B7F1900039120045
:102457001EE0FC90E60012001EECF078597401268D
:10246700F6500418E436F650CF755900755800AE8B
:1024770058AF5974FFC39F74019E402475B7A57563
:10248700B7F190023912001EE0FC90E80012001E1E
:10249700ECF07859740126F6500418E436F650CF5C
:1024A700755900755800AE58AF5974FFC39F740132
:1024B7009E402475B7A575B7F190043912001EE048
:1024C700FC90EA0012001EECF07859740126F650D1
:1024D7000418E436F650CF755900755800AE58AF5A
:1024E7005974FFC39F74019E402475B7A575B7F152
:1024F70090063912001EE0FC90EC0012001EECF072
:102507007859740126F6500418E436F650CF758FC3
:102517000075F51175B62075D940D2AF743A90079A
:1025270039F02290083BE0B4AA028003022667C272
:10253700AF75D90075B62275F522758F0375B7A5E6
:1025470075B7F1740090DE00F075B7A575B7F17433
:102557000090E000F075B7A575B7F1740090E20040
:10256700F075B7A575B7F1740090E400F0758F01A9
:10257700755900755800AE58AF5974FFC39F740161
:102587009E402475B7A575B7F190003912001EE07B
:10259700FC90DE0012001EECF07859740126F6500C
:1025A7000418E436F650CF755900755800AE58AF89
:1025B7005974FFC39F74019E402475B7A575B7F181
:1025C70090023912001EE0FC90E00012001EECF0B1
:1025D7007859740126F6500418E436F650CF755929
:1025E70000755800AE58AF5974FFC39F74019E40E1
:1025F7002475B7A575B7F190043912001EE0FC9059
:10260700E20012001EECF07859740126F650041807
:10261700E436F650CF755900755800AE58AF597467
:10262700FFC39F74019E402475B7A575B7F1900647
:102637003912001EE0FC90E40012001EECF07859FD
:10264700740126F6500418E436F650CF758F0075DE
:10265700F51175B62075D940D2AF743A900739F0A5
:102667002290083BE0B4AA0280030227A5C2AF75F7
:10267700D90075B62275F522758F0375B7A575B79D
:10268700F1740090D600F075B7A575B7F174009096
:10269700D800F075B7A575B7F1740090DA00F0753A
:1026A700B7A575B7F1740090DC00F0758F01755907
:1026B70000755800AE58AF5974FFC39F74019E4010
:1026C7002475B7A575B7F190003912001EE0FC908C
:1026D700D60012001EECF07859740126F650041843
:1026E700E436F650CF755900755800AE58AF597497
:1026F700FFC39F74019E402475B7A575B7F190027B
:102707003912001EE0FC90D80012001EECF0785938
:10271700740126F6500418E436F650CF7559007543
:102727005800AE58AF5974FFC39F74019E4024757B
:10273700B7A575B7F190043912001EE0FC90DA00D6
:1027470012001EECF07859740126F6500418E4368E
:10275700F650CF755900755800AE58AF5974FFC37E
:102767009F74019E402475B7A575B7F1900639127D
:10277700001EE0FC90DC0012001EECF0785974019A
:1027870026F6500418E436F650CF758F0075F5110C
:1027970075B62075D940D2AF743A900739F022C286
:1027A700AF75D90075F522755900755800AE58AF49
:1027B7005974FFC39F74019E401F90EE0012001EC4
:1027C700E493FC90003912001EECF078597401264E
:1027D700F6500418E436F650D4755900755800AE13
:1027E70058AF5974FFC39F74019E401F90F00012A9
:1027F700001EE493FC90023912001EECF078597425
:102807000126F6500418E436F650D4755900755869
:1028170000AE58AF5974FFC39F74019E401F90F2DA
:102827000012001EE493FC90043912001EECF078AD
:1028370059740126F6500418E436F650D475590039
:10284700755800AE58AF5974FFC39F74019E401F5F
:1028570090F40012001EE493FC90063912001EEC5F
:10286700F07859740126F6500418E436F650D475FA
:10287700F51175D940D2AF740090006DF0740190D6
:102887000043F0743A900739F022C2AF75D900754A
:10289700F522755900755800AE58AF5974FFC39F9C
:1028A70074019E401F90E60012001EE493FC900006
:1028B7003912001EECF07859740126F6500418E41A
:1028C70036F650D4755900755800AE58AF5974FF95
:1028D700C39F74019E401F90E80012001EE493FC02
:1028E70090023912001EECF07859740126F6500454
:1028F70018E436F650D4755900755800AE58AF59DC
:1029070074FFC39F74019E401F90EA0012001EE4EB
:1029170093FC90043912001EECF07859740126F6E6
:10292700500418E436F650D4755900755800AE585F
:10293700AF5974FFC39F74019E401F90EC001200B3
:102947001EE493FC90063912001EECF078597401CE
:1029570026F6500418E436F650D475F51175D940AB
:10296700D2AF740090006DF07402900043F0743A97
:10297700900739F022C2AF75D90075F52275590055
:10298700755800AE58AF5974FFC39F74019E401F1E
:1029970090DE0012001EE493FC90003912001EEC3A
:1029A700F07859740126F6500418E436F650D475B9
:1029B7005900755800AE58AF5974FFC39F74019EF4
:1029C700401F90E00012001EE493FC9002391200B1
:1029D7001EECF07859740126F6500418E436F650C8
:1029E700D4755900755800AE58AF5974FFC39F741A
:1029F700019E401F90E20012001EE493FC900439F0
:102A070012001EECF07859740126F6500418E436CB
:102A1700F650D4755900755800AE58AF5974FFC3B6
:102A27009F74019E401F90E40012001EE493FC90E7
:102A3700063912001EECF07859740126F650041876
:102A4700E436F650D475F51175D940D2AF740090BD
:102A5700006DF07403900043F0743A900739F02248
:102A6700C2AF75D90075F522755900755800AE5873
:102A7700AF5974FFC39F74019E401F90D600120088
:102A87001EE493FC90003912001EECF07859740193
:102A970026F6500418E436F650D4755900755800D8
:102AA700AE58AF5974FFC39F74019E401F90D80062
:102AB70012001EE493FC90023912001EECF07859C4
:102AC700740126F6500418E436F650D4755900758B
:102AD7005800AE58AF5974FFC39F74019E401F90B2
:102AE700DA0012001EE493FC90043912001EECF089
:102AF7007859740126F6500418E436F650D47559FF
:102B070000755800AE58AF5974FFC39F74019E40BB
:102B17001F90DC0012001EE493FC90063912001E81
:102B2700ECF07859740126F6500418E436F650D4C0
:102B370075F51175D940D2AF740090006DF074042B
:102B4700900043F0743A900739F022E56864046016
:102B570006E59964FF60028031A20D4004D20D8022
:102B670027E568600874E62568900024F0E567604B
:102B77000874F02567900024F0E568B4010280FE30
:102B8700756800756700C20D8002C20DE568903850
:102B97008CF8282873756800E599B4FF03756701F9
:102BA700E599B4FE03756702E599B4FD03756703FC
:102BB700E599B4FC03756704E599B4FA03756705ED
:102BC700E599B4FB067568011205B2E599B4F906F3
:102BD7007568041205B2E599B4F7411205B2C29CB3
:102BE70074AB90083BF012220374AA90083BF0E5FF
:012BF7004994
:03388C00022B9C70
:102BF8009038ECF828287380121222AE800D122328
:0B2C0800EC800812252A8003122668C9
:0F38EC00022BFF022C01022C06022C0B022C10C7
:102C130090083BE4F0D29C7568007567007599F7DE
:102C2300E599D394E54007E599C394F040028016F3
:102C33008599697568027E017F00E569C394E61290
:102C43003E568E5E8F5F900839E4F0A3F0E599D38A
:102C530094C44007E599C394E640028028859969A6
:102C630075680374E5C39569F55F755E00AE5EAF85
:102C73005F903D6712002EE493F874019390083936
:102C8300C8F0A3C8F0D299022F67900839E0FEA3D9
:102C9300E0FF90003912001EE599F0900839120008
:102CA3000E900839E0FEA3E0FFEFB40106EEB4078F
:102CB300028003022D75900739E0B43C02800302C1
:102CC3002D751207B0A206B35005A207B3400280C8
:102CD30053C29C120088120282900125E090085A88
:102CE300F0900126E090085BF0900127E090085CEB
:102CF300F074AB90083BF012220374AA90083BF0E7
:022D0300E549A0
:03388F00022C8D7B
:102D05009038FBF828287380121222AE800D12230A
:0B2D1500EC800812252A8003122668BB
:0F38FB00022D0C022D0E022D13022D18022D1D71
:102D200090083BE4F08043C29C1220177400900886
:102D30005AF0740090085BF0740090085CF074AB7B
:102D400090083BF012220374AA90083BF01222AEC6
:102D50001223EC12252A122668D29C7599FB746402
:102D6000F50975080012214D80FED29C756800752A
:102D700067007599FB022F67900839E0FEA3E0FF1A
:102D8000EF4E700685995D755C00900839E0FEA3F2
:102D9000E0FF74016F4E701BAC5CAD5DAA5EAB5F73
:102DA000ED2BFBEC3AFA8A068B0790003912001ED5
:102DB000E599F090083912000E900839E0FEA3E082
:102DC000FF74026F4E700C1202828569997568005B
:102DD000756700022F67900839E0FEA3E0FF9000BE
:102DE0003912001EE599F090083912000E9008394A
:102DF000E0FEA3E0FFAC5EAD5F8F028E038C068D1C
:102E000007903D9F12002EE493F9740193FEEAD3DC
:102E10009EEB994009856999756800756700022FD6
:102E200067900839E0FEA3E0FF90003912001EE52C
:102E300099F090083912000E900839E0FEA3E0FFE7
:102E4000EFB40006EEB401028003022F6790001871
:102E5000E0D394C7400B900018E0C394C8F56A8093
:102E60001A900018E0D39463400B900018E0C394CC
:102E700064F56A8006900018E0F56AE56A75F0026C
:102E8000A4FFAEF08F66EF900039123E6EEFFCE0CB
:102E9000FDEC90003C123E6EEDFCE0FDEC2DB56AC1
:102EA000028003022F580FEF900039123E6EE56644
:102EB000FFE0FCEF90003D123E6EECFFE0FCEFC344
:102EC0009CB56A028003022F58E56690003B123ED3
:102ED0006EE566FFE0FCEF90003E123E6EECFFE018
:102EE000FCEF2CB56A72E56690003F123E6EE0C3BF
:102EF000956A900878F0E566900040123E6EE0C357
:102F0000956A900879F0E566900043123E6EE0C342
:102F1000956A90087AF0E566900044123E6EE0C330
:102F2000956A90087BF0E566900045123E6EE0C31E
:102F3000956A90087CF0E566900046123E6EE0C30C
:102F4000956A90087DF01221797599F97464F509F4
:102F500075080012214D80FE7599FF7464F509759E
:072F6000080012214D80FE64
:09389200022D78022DD6022E2130
:102F670022E56790389BF82828730230A890083923
:102F7700E0FEA3E0FF90000812001EE0F59990081C
:102F87003912000E900839E0FEA3E0FF741C6F4E63
:102F970070037567000230A88550990230A8900821
:102FA70039E0FEA3E0FF90003912001EE0F599EF2B
:102FB700B40107EEB4070375670090083912000ED5
:072FC7000230A890083AE077
:0F389B00022F71022F74022F9F022FA5022FCA36
:102FCE0090390AF828287385249902309D852A990C
:102FDE0002309D853B9902309D853D9902309D853D
:102FEE00449902309D854F9902309D854899023053
:102FFE009D85499902309D756B00900054E07006D6
:10300E00900053E060028016A2A44006E56B4404D3
:10301E00F56BA2A54006E56B4402F56B801A900095
:10302E0034E0B40106E56B4410F56B900033E0B468
:10303E000106E56B4420F56BA203B34006E56B4435
:10304E0001F56BA205B34006E56B4408F56B856B85
:10305E0099803CA20EB340077599FAC20E8017A252
:10306E000AB3400575990F800B900024E0F59990F6
:10307E000024E4F0C20A8017853A9980128540999F
:0F308E00800D856C9980087599FC80037567002B
:10390A00022FD5022FDB022FE1022FE7022FED0251
:10391A002FF3022FF9022FFF023005023061023025
:0D392A008602308B02309002309502309AF8
:0B309D0090083912000E800312023B65
:0338AA000230A544
:1030A80022E50875F003A4FFAEF0EF241AF509E550
:1030B8000904F50AE5092402F50BE509900039121F
:1030C8003E6EE09038ADF82828738021852464800E
:1030D8001C852A648017853B648012853D64800DB9
:0D30E8008544648008854864800385496440
:1038AD000230D20230D40230D90230DE0230E302CF
:0838BD0030E80230ED0230F2A8
:1030F500E50A900039123E6EE50BFEE0FFEE90000A
:1031050039123E6EEFFEE0FFEED39F40030232031D
:10311500E509900039123E6EE0D394044051E50A6A
:10312500900039123E6EE0D39564500EE50B900089
:1031350039123E6EE0C395645002800AE508F50C2D
:10314500D39210120048E50A900039123E6EE0D382
:103155009564500EE50B900039123E6EE0C3956400
:10316500500AE508F50CC39210120048023200E53A
:1031750009900039123E6EE0B40432E50B90003937
:10318500123E6EE0C39564500AE508F50CD3921023
:10319500120048E50A900039123E6EE0D39564406E
:1031A5000AE508F50CC39210120048804EE50A9016
:1031B5000039123E6EE0C39564500EE50B90003960
:1031C500123E6EE0D395645002800AE508F50CD3F3
:1031D5009210120048E50A900039123E6EE0D39530
:1031E50064500EE50B900039123E6EE0C3956450B5
:1031F5000AE508F50CC392101200480232EEE50903
:10320500900039123E6EE0D394044051E50A9000D7
:1032150039123E6EE0C39564400EE50B90003912FD
:103225003E6EE0D395644002800AE508F50CC39232
:1032350010120048E50A900039123E6EE0C395640D
:10324500400EE50B900039123E6EE0D39564400ABE
:10325500E508F50CD392101200480232EEE509900C
:103265000039123E6EE0B40432E50A900039123E90
:103275006EE0C39564500AE508F50CC39210120080
:1032850048E50B900039123E6EE0D39564400AE59F
:1032950008F50CD39210120048804EE50A900039CB
:1032A500123E6EE0C39564400EE50B900039123E68
:1032B5006EE0D39564400AE508F50CD39210120030
:1032C50048E50A900039123E6EE0D39564400EE55C
:1032D5000B900039123E6EE0C395644002800AE50A
:1032E50008F50CC3921012004822E56D9038C5F818
:1032F5002828730238797E017F00E5BE123E56E527
:10330500BD2FFF50010E8E5A8F5B900065E0B40112
:103315000F7E0F7FFFAC5AAD5B1200038E5A8F5B99
:10332500900064E0B40245AE5AAF5B900000E0FC4B
:10333500A3E0FDEDD39FEC9E400A900000E55AF016
:10334500A3E55BF0AE5AAF5B900002E0FCA3E0FDA5
:10335500EFD39DEE9C400A900002E55AF0A3E55B91
:10336500F0AE5AAF5B7404123E488F3B900064E0A8
:103375007058AE5AAF5B900000E0FCA3E0FDEFD3C0
:103385009DEE9C40091200038E5A8F5B8006755B8B
:1033950000755A00900063E0700674FF900063F0BA
:1033A500AE5AAF5B7410123E56900063E08E048FE8
:1033B50005FF123E388C5A8D5B7400D39D74019CB9
:1033C5004005855B3B8003753BFFE53B75F00AA433
:1033D500FFAEF074198E048F05FF123E388D3CED5B
:1033E5002561FFAE6050010E7401123E488F3C8589
:1033F5003C61756000EFD394624003753C629000B8
:103405005DE07006900051E060028006756D050272
:1034150032EF75BB170238790238797E017F00E5F6
:10342500BE123E56E5BD2FFF50010E8E5A8F5B90A2
:10343500005DE0B4017AE56345626025AC62AD6389
:103445001DBDFF011C8F028E038C068D0790393739
:1034550012002EE493FE740193FFEFC39AEE9B4096
:103465000280057862123E80AE62AF6374B3BE001F
:1034750021D39F401DAC5AAD5B0FBF00010E9039A3
:103485003712002EE493FE740193FFEDC39FEC9E6B
:1034950040028005786212003FAE62AF6390005F24
:1034A500E0123E5674648E048F05FF123E388D3D42
:1034B500E570B40129AE5AAF5BEFD39400EE9408E2
:1034C500400F900051E0B40104C2058002D205808E
:1034D5000D900051E0B40104D2058002C20575BB10
:1034E500160238790238797E017F00E5BE123E5614
:1034F500E5BD2FFF50010E8E5A8F5B90005DE0B445
:10350500027AE56345626025AC62AD631DBDFF01CE
:103515001C8F028E038C068D07903AA112002EE4B3
:1035250093FE740193FFEFC39AEE9B4002800578EA
:1035350062123E80AE62AF6374B3BE0021D39F407A
:103545001DAC5AAD5B0FBF00010E903AA112002EC3
:10355500E493FE740193FFEDC39FEC9E400280054A
:10356500786212003FAE62AF6390005FE0123E5694
:1035750074648E048F05FF123E388D3DE570B402EC
:1035850029AE5AAF5BEFD39400EE9408400F90003C
:1035950051E0B40104C2058002D205800D900051AE
:1035A500E0B40104D2058002C20590005DE070031D
:1035B500753D00900051E07002C20575BB1F0238D1
:1035C500790238797E017F00E5BE123E56E5BD2FB2
:1035D500FF50010E8E5A8F5B7409123E5674E68EAB
:1035E500048F05FF123E388C398D3AE56E2DFD505E
:1035F500010C74018C068D07123E488E398F3A8571
:103605003A6E75BB190238790238797E017F00E57B
:10361500BE123E56E5BD2FFF50010E8E5A8F5B74CC
:1036250004123E488F4090006BE0B4010280030213
:1036350036E6756600756600E566D39407400302B5
:1036450036DCE56690002B123E6EE0D39540501AAD
:10365500E56690002B123E6EE0F4042540FEE5661B
:1036650090087E123E6EEEF08017E56690002B12F4
:103675003E6EE0C39540FEE56690087E123E6EEE16
:10368500F0E566C39404400990006FE0C395665069
:103695003BE5666029E56690087E123E6EFEE0FF1A
:1036A500EE900886E0D39F4013E56690087E123EB3
:1036B5006EE0900886F0E566900887F0800E900829
:1036C5007EE0900886F07400900887F078667401B3
:1036D50026F6400302363D900887E0F4042408F5F9
:1036E5004890006BE0D394014033E540D3946E409D
:1036F50004D20F8002C20F75480590006BE0B4023A
:1037050005A20FB34002800375480790006BE0B433
:103715000306A20FB3B340028003754807E56F6542
:10372500486008E54404F54585486FE548B4070851
:10373500E5B54480F5B58006E5B5547FF5B5E548B2
:1037450064066005E548B40808E5B54410F5B5809C
:1037550006E5B554EFF5B575BB130238790238792E
:103765007E017F00E5BE123E56E5BD2FFF50010EDE
:103775008E5A8F5B7404123E488F6C90006CE0B4D7
:1037850002028003023874756600756600E566D32B
:1037950094034003023821E566900027123E6EE04F
:1037A500D3956C501AE566900027123E6EE0F4043E
:1037B500256CFEE566900888123E6EEEF08017E5F2
:1037C50066900027123E6EE0C3956CFEE566900894
:1037D50088123E6EEEF0E5666029E566900888126F
:1037E5003E6EFEE0FFEE90088CE0D39F4013E56649
:1037F500900888123E6EE090088CF0E56690088D82
:10380500F0800E900888E090088CF0740090088D88
:10381500F07866740126F6400302379290006DE059
:10382500704DE52A45296036E549C39403500A9051
:10383500088DE004C394034002800790088DE004DE
:10384500F549E549D39402400A90088DE004D394E4
:10385500025002800790088DE004F5498011900818
:103865008DE004F549E549D3940440037549017594
:04387500BB188000FC
:1038C5000232F80232FB02341D0234200234E902CE
:1038D50034EC0235C60235C902360D023610023700
:0738E5006202376502387929
:10387900E56D75F00284AFF07E00EF4E7002D2EC78
:03388900056D22A8
:093E6E002582F582500205832231
:10002E00EF2F500205832582F582E5833E2EF58360
:01003E00229F
:08000300C3EF9DFFEE9CFE22FD
:08003F000806B60002180622B3
:0D000E00A3E004F07006123E64E004F0224E
:083E80000816B6FF0218162215
:0E3E4800048007C3CE13CECF13CFD5E0F622F1
:103C8600BC000FBE0008ED8FF084FFADF022E4FE0D
:103C9600FF22BE000DEF60FE54F0606F20E70302C6
:103CA6003D3CEAC0E0EBC0E078017A0075F001EE39
:103CB60020E710EF25E0FFEE33FE0AC5F023C5F03E
:103CC60030E7F0EA5407F9096A7A007B00600108D8
:103CD600C3EC9E40167004ED9F4010ED9FFDEC9ED8
:103CE600FCE5F0CA4ACA03F5F08005E5F003F5F0F5
:103CF600C3EE13FEEF13FFD9D77908CACBCAD8D0C3
:103D0600EAFEEBFFD0E0FBD0E0FA22EC8FF084FC79
:103D1600ED54F045F0C48FF084FEEDC454F045F048
:103D2600C48FF084FDEEC4FE54F02DFFEE540F3C1C
:103D3600FEADF07C0022790078008FF0EC7E082042
:103D4600E70DC3CD33CD33C933C9C833C8DEF084DC
:103D560049F9E5F08FF0BE00E6FD7C00E9FFE8FEDC
:013D6600223A
:0E3E5600F88FF0A4FFE5F0CE88F0A42EFE2237
:103E2800600D782B023E32007830D8FED5E0F822BB
:103E3800EEC0E07E00123C86EFFDEEFCD0E0FE22F4
:03000B00023DD7DC
:03001B00023DF2B1
:03002B00023E0D85
:03000000023E7746
:093E770075817175D0000207C2CB
:0B001E00E5822FF582E5833EF583228A
:0A3E64000582D58202158315822223
:103DD700C0E0C0F0C083C082C0D075D0001207B762
:103DE700D0D0D082D083D0F0D0E032C0E0C0F0C0D5
:103DF70083C082C0D075D0001207BAD0D0D082D08D
:103E070083D0F0D0E032C0E0C0F0C083C082C0D021
:103E170075D0001207BDD0D0D082D083D0F0D0E0CB
:013E27003268
:00000001FF
